 ddi_powervr

 Timestamp is 4acad54e (Tue Oct 06 14:27:42 2009)

 Preferred load address is 10000000

 Start         Length     Name                   Class
 0001:00000000 00000004H .CRT$XCA                CODE
 0001:00000004 00000004H .CRT$XCU                CODE
 0001:00000008 00000004H .CRT$XCZ                CODE
 0001:0000000c 00000004H .CRT$XIA                CODE
 0001:00000010 00000004H .CRT$XIZ                CODE
 0001:00000014 00000004H .CRT$XPA                CODE
 0001:00000018 00000004H .CRT$XPZ                CODE
 0001:0000001c 00000004H .CRT$XTA                CODE
 0001:00000020 00000004H .CRT$XTZ                CODE
 0001:00000030 00001a68H .rdata                  CODE
 0001:00001a98 00000028H .rdata$debug            CODE
 0001:00001ac0 00029378H .text                   CODE
 0001:0002ae38 00000030H .text$yc                CODE
 0001:0002ae68 000000d4H .xdata                  CODE
 0001:0002af3c 00000014H .idata$2                CODE
 0001:0002af50 00000014H .idata$3                CODE
 0001:0002af64 000000e8H .idata$4                CODE
 0001:0002b04c 0000000cH .idata$6                CODE
 0001:0002b060 0000005eH .edata                  CODE
 0002:00000000 000000e8H .idata$5                DATA
 0002:000000e8 0000c1a0H .data                   DATA
 0002:0000c288 00003eb4H .bss                    DATA
 0003:00000000 00000d90H .pdata                  DATA

  Address         Publics by Value              Rva+Base       Lib:Object

 0000:00000000       ___safe_se_handler_count   00000000     <absolute>
 0000:00000000       ___safe_se_handler_table   00000000     <absolute>
 0001:00000000       __xc_a                     10001000     corelib0:crt0init.obj
 0001:00000008       __xc_z                     10001008     corelib0:crt0init.obj
 0001:0000000c       __xi_a                     1000100c     corelib0:crt0init.obj
 0001:00000010       __xi_z                     10001010     corelib0:crt0init.obj
 0001:00000014       __xp_a                     10001014     corelib0:crt0init.obj
 0001:00000018       __xp_z                     10001018     corelib0:crt0init.obj
 0001:0000001c       __xt_a                     1000101c     corelib0:crt0init.obj
 0001:00000020       __xt_z                     10001020     corelib0:crt0init.obj
 0001:0000004c       ??_C@_1CG@OEHAIELG@?$AAI?$AAO?$AAC?$AAT?$AAL?$AA_?$AAP?$AAO?$AAW?$AAE?$AAR?$AA_?$AAQ?$AAU?$AAE?$AAR?$AAY?$AA?6?$AA?$AA@ 1000104c     control.obj
 0001:00000078       ??_C@_1FO@BHOOHNF@?$AAU?$AAn?$AAa?$AAb?$AAl?$AAe?$AA?5?$AAt?$AAo?$AA?5?$AAi?$AAn?$AAi?$AAt?$AAi?$AAa?$AAl?$AAi?$AAz?$AAe?$AA?5?$AAS?$AAG?$AAX?$AA?5?$AAd?$AAi?$AAs?$AAp?$AAl?$AAa?$AAy@ 10001078     init.obj
 0001:000000d8       ??_C@_1EE@OMNLEFOF@?$AAU?$AAn?$AAa?$AAb?$AAl?$AAe?$AA?5?$AAt?$AAo?$AA?5?$AAd?$AAe?$AAs?$AAt?$AAr?$AAo?$AAy?$AA?5?$AAd?$AAe?$AAv?$AAi?$AAc?$AAe?$AA?5?$AAc?$AAo?$AAn?$AAt?$AAe?$AAx?$AAt@ 100010d8     init.obj
 0001:000001c0       ??_C@_1BC@PGJONGEG@?$AAB?$AAi?$AAt?$AAD?$AAe?$AAp?$AAt?$AAh?$AA?$AA@ 100011c0     mode.obj
 0001:000001d4       ??_C@_1O@BLHDEIAD@?$AAH?$AAe?$AAi?$AAg?$AAh?$AAt?$AA?$AA@ 100011d4     mode.obj
 0001:000001e4       ??_C@_1M@NLLLJLND@?$AAW?$AAi?$AAd?$AAt?$AAh?$AA?$AA@ 100011e4     mode.obj
 0001:000001f0       ??_C@_1DA@JKODHAGA@?$AAD?$AAr?$AAi?$AAv?$AAe?$AAr?$AAs?$AA?2?$AAD?$AAi?$AAs?$AAp?$AAl?$AAa?$AAy?$AA?2?$AAP?$AAo?$AAw?$AAe?$AAr?$AAV?$AAR?$AA?$AA@ 100011f0     mode.obj
 0001:00000220       ??_C@_1GI@LBPPMOKF@?$AA?$HL?$AA?$CF?$AA0?$AA8?$AAl?$AAX?$AA?9?$AA?$CF?$AA0?$AA4?$AAX?$AA?9?$AA?$CF?$AA0?$AA4?$AAX?$AA?9?$AA?$CF?$AA0?$AA2?$AAX?$AA?$CF?$AA0?$AA2?$AAX?$AA?9?$AA?$CF?$AA0?$AA2?$AAX?$AA?$CF?$AA0@ 10001220     power.obj
 0001:00000288       ??_C@_1CE@LGAKADBG@?$AAD?$AAi?$AAs?$AAp?$AAl?$AAa?$AAy?$AAP?$AAo?$AAw?$AAe?$AAr?$AAC?$AAl?$AAa?$AAs?$AAs?$AA?$AA@ 10001288     power.obj
 0001:000002b0       ??_C@_1EO@BHDHHEGO@?$AA?$HL?$AAE?$AAB?$AA9?$AA1?$AAC?$AA7?$AAC?$AA9?$AA?9?$AA8?$AAB?$AAF?$AA6?$AA?9?$AA4?$AAa?$AA2?$AAd?$AA?9?$AA9?$AAA?$AAB?$AA8?$AA?9?$AA6?$AA9?$AA7?$AA2?$AA4?$AAE?$AAE@ 100012b0     power.obj
 0001:00000300       ??_C@_1CG@BEPCNIEH@?$AAS?$AAy?$AAs?$AAt?$AAe?$AAm?$AA?2?$AAG?$AAD?$AAI?$AA?2?$AAD?$AAr?$AAi?$AAv?$AAe?$AAr?$AAs?$AA?$AA@ 10001300     power.obj
 0001:00000328       ??_C@_1M@FIJHFMPA@?$AAA?$AAN?$AAG?$AAL?$AAE?$AA?$AA@ 10001328     rotate.obj
 0001:00000334       ??_C@_1CI@PNCEGBJC@?$AAS?$AAY?$AAS?$AAT?$AAE?$AAM?$AA?2?$AAG?$AAD?$AAI?$AA?2?$AAR?$AAO?$AAT?$AAA?$AAT?$AAI?$AAO?$AAN?$AA?$AA@ 10001334     rotate.obj
 0001:00000360       ??_7SGX@@6B@               10001360     sgxmain.obj
 0001:000003e0       ??_7GPESurf@@6B@           100013e0     surf.obj
 0001:000003e4       ??_7SGXSurf@@6B@           100013e4     surf.obj
 0001:000003e8       ??_C@_1DK@IFOPGNGH@?$AAA?$AAl?$AAl?$AAo?$AAc?$AAS?$AAu?$AAr?$AAf?$AAa?$AAc?$AAe?$AA?5?$AA?9?$AA?5?$AAO?$AAu?$AAt?$AA?5?$AAo?$AAf?$AA?5?$AAM?$AAe?$AAm?$AAo?$AAr?$AAy?$AA?$AA@ 100013e8     surf.obj
 0001:00000428       g_NullBlendFunction        10001428     gpe:ddi_if.obj
 0001:000004ac       ??_C@_17BJMBELJK@?$AAG?$AAP?$AAE?$AA?$AA@ 100014ac     gpe:ddi_if.obj
 0001:000004b4       EGPEFormatToBpp            100014b4     gpe:gpe.obj
 0001:000004d8       EGPEFormatToIFormat        100014d8     gpe:gpe.obj
 0001:000004fc       IFormatToEGPEFormat        100014fc     gpe:gpe.obj
 0001:00000528       ??_7GPE@@6B@               10001528     gpe:gpe.obj
 0001:000005a4       ??_C@_1BM@OHJNPODK@?$AAA?$AAs?$AAp?$AAe?$AAc?$AAt?$AAR?$AAa?$AAt?$AAi?$AAo?$AAX?$AAY?$AA?$AA@ 100015a4     gpe:gpe.obj
 0001:000005c0       ??_C@_1BK@GPCKCPMK@?$AAA?$AAs?$AAp?$AAe?$AAc?$AAt?$AAR?$AAa?$AAt?$AAi?$AAo?$AAY?$AA?$AA@ 100015c0     gpe:gpe.obj
 0001:000005dc       ??_C@_1BK@NHJGEIKP@?$AAA?$AAs?$AAp?$AAe?$AAc?$AAt?$AAR?$AAa?$AAt?$AAi?$AAo?$AAX?$AA?$AA@ 100015dc     gpe:gpe.obj
 0001:000005f8       ??_C@_1BO@ONBCMHFO@?$AAL?$AAo?$AAg?$AAi?$AAc?$AAa?$AAl?$AAP?$AAi?$AAx?$AAe?$AAl?$AAs?$AAY?$AA?$AA@ 100015f8     gpe:gpe.obj
 0001:00000618       ??_C@_1BO@FFKOKADL@?$AAL?$AAo?$AAg?$AAi?$AAc?$AAa?$AAl?$AAP?$AAi?$AAx?$AAe?$AAl?$AAs?$AAX?$AA?$AA@ 10001618     gpe:gpe.obj
 0001:00000638       ??_C@_1BK@HNDINEGH@?$AAV?$AAe?$AAr?$AAt?$AAi?$AAc?$AAa?$AAl?$AAS?$AAi?$AAz?$AAe?$AA?$AA@ 10001638     gpe:gpe.obj
 0001:00000654       ??_C@_1BO@CPEMBNKP@?$AAH?$AAo?$AAr?$AAi?$AAz?$AAo?$AAn?$AAt?$AAa?$AAl?$AAS?$AAi?$AAz?$AAe?$AA?$AA@ 10001654     gpe:gpe.obj
 0001:00000a78       ??_C@_15MAOEGKJF@?$AA?$CF?$AAS?$AA?$AA@ 10001a78     srvclkm:srvclient_wince.obj
 0001:00001134       ??_C@_1M@DMCDIEDK@?$AAP?$AAK?$AAM?$AA1?$AA?3?$AA?$AA@ 10002134     srvclkm:pvr_bridge_clientkm.obj
 0001:00001ac0       ?UnRotate@SGX@@AAAXPAU_RECTL@@PAVSGXSurf@@@Z 10002ac0 f   bltfuncs.obj
 0001:00001b5c       ?ClippedBlt@SGX@@AAAJPAUGPEBltParms@@PAU_PVR2DBLTINFO@@@Z 10002b5c f   bltfuncs.obj
 0001:00001d88       ?BltClear@SGX@@AAAJPAUGPEBltParms@@@Z 10002d88 f   bltfuncs.obj
 0001:00001dd0       ?BltSet@SGX@@AAAJPAUGPEBltParms@@@Z 10002dd0 f   bltfuncs.obj
 0001:00001e18       ?BltFillSolidColor@SGX@@AAAJPAUGPEBltParms@@@Z 10002e18 f   bltfuncs.obj
 0001:00001e8c       ?BltCopySource@SGX@@AAAJPAUGPEBltParms@@@Z 10002e8c f   bltfuncs.obj
 0001:00001ecc       ?BltAndSource@SGX@@AAAJPAUGPEBltParms@@@Z 10002ecc f   bltfuncs.obj
 0001:00001f0c       ?BltInvertSource@SGX@@AAAJPAUGPEBltParms@@@Z 10002f0c f   bltfuncs.obj
 0001:00001f4c       ?BltInvertDest@SGX@@AAAJPAUGPEBltParms@@@Z 10002f4c f   bltfuncs.obj
 0001:00001f8c       ?isOverlappedBltParameter@@YA_NPAUGPEBltParms@@@Z 10002f8c f   bltfuncs.obj
 0001:00002010       ?BltPrepare@SGX@@UAAJPAUGPEBltParms@@@Z 10003010 f   bltfuncs.obj
 0001:00002454       ?BltComplete@SGX@@UAAJPAUGPEBltParms@@@Z 10003454 f   bltfuncs.obj
 0001:00002474       ?WaitForNotBusy@SGX@@UAAXXZ 10003474 f   bltfuncs.obj
 0001:00002498       ?IsBusy@SGX@@UAAHXZ        10003498 f   bltfuncs.obj
 0001:000024d0       DrvGetMasks                100034d0 f   control.obj
 0001:000024e0       ?DrvEscape@SGX@@UAAKPAU_SURFOBJ@@KKPAXK1@Z 100034e0 f   control.obj
 0001:000027bc       ?CursorOn@SGX@@QAAXXZ      100037bc f   cursor.obj
 0001:00002a60       ?CursorOff@SGX@@QAAXXZ     10003a60 f   cursor.obj
 0001:00002bd4       ?SetPointerShape@SGX@@UAAJPAVGPESurf@@0HHHH@Z 10003bd4 f   cursor.obj
 0001:00002cec       ?MovePointer@SGX@@UAAJHH@Z 10003cec f   cursor.obj
 0001:00002d50       ?InitializeHardware@SGX@@AAAHXZ 10003d50 f   init.obj
 0001:00002ec4       ?DeInitializeHardware@SGX@@AAAHXZ 10003ec4 f   init.obj
 0001:00002f0c       ?GetGameXInfo@SGX@@QAAHKKPAXK0@Z 10003f0c f   gapi.obj
 0001:000030cc       ?WrappedEmulatedLine@SGX@@QAAJPAUGPELineParms@@@Z 100040cc f   line.obj
 0001:000032e4       ?Line@SGX@@UAAJPAUGPELineParms@@W4EGPEPhase@@@Z 100042e4 f   line.obj
 0001:0000331c       ?GetModeInfo@SGX@@UAAJPAUGPEMode@@H@Z 1000431c f   mode.obj
 0001:00003354       ?NumModes@SGX@@UAAHXZ      10004354 f   mode.obj
 0001:0000335c       ?PVR2DFormatToGPEFormat@SGX@@AAA?AW4EGPEFormat@@W4PVR2DFORMAT@@@Z 1000435c f   mode.obj
 0001:000033a4       ?PVR2DFormatToBpp@SGX@@AAAHW4PVR2DFORMAT@@@Z 100043a4 f   mode.obj
 0001:000033ec       ?SetPalette@SGX@@UAAJPBUtagPALETTEENTRY@@GG@Z 100043ec f   mode.obj
 0001:00003410       ?InitializeModes@SGX@@AAAHXZ 10004410 f   mode.obj
 0001:00003618       ?DeInitializeModes@SGX@@AAAHXZ 10004618 f   mode.obj
 0001:0000365c       ?GetGraphicsCaps@SGX@@UAAKXZ 1000465c f   mode.obj
 0001:00003684       ?getColorDepth@SGX@@QAAHXZ 10004684 f   mode.obj
 0001:000036fc       ?PrimarySurfaceSetMode@SGX@@AAAHH@Z 100046fc f   mode.obj
 0001:000037cc       ?SetMode@SGX@@UAAJHPAPAUHPALETTE__@@@Z 100047cc f   mode.obj
 0001:000038e0       ?VideoToPmPowerState@@YA?AW4_CEDEVICE_POWER_STATE@@W4_VIDEO_POWER_STATE@@@Z 100048e0 f   power.obj
 0001:00003a0c       ?AdvertisePowerInterface@SGX@@AAAHXZ 10004a0c f   power.obj
 0001:00003b2c       ?GetRotateModeFromReg@SGX@@QAAHXZ 10004b2c f   rotate.obj
 0001:00003bf0       ?SetRotateParams@SGX@@QAAXXZ 10004bf0 f   rotate.obj
 0001:00003c44       ?DynRotate@SGX@@QAAJH@Z    10004c44 f   rotate.obj
 0001:00003ce0       ?RegisterDDHALAPI@@YAXXZ   10004ce0 f   sgxmain.obj
 0001:00003ce4       DrvEnableDriver            10004ce4 f   sgxmain.obj
 0001:00003ce8       ??0SGX@@QAA@PAH@Z          10004ce8 f   sgxmain.obj
 0001:00003d7c       ?GetPhysicalVideoMemory@SGX@@UAAXPAK0@Z 10004d7c f   sgxmain.obj
 0001:00003da0       ?InVBlank@SGX@@UAAHXZ      10004da0 f   sgxmain.obj
 0001:00003dc4       DisplayInit                10004dc4 f   sgxmain.obj
 0001:00003e40       GetGPE                     10004e40 f   sgxmain.obj
 0001:00003ebc       ??_GSGX@@UAAPAXI@Z         10004ebc f i sgxmain.obj
 0001:00003ebc       ??_ESGX@@UAAPAXI@Z         10004ebc f i sgxmain.obj
 0001:00003ef4       ??0GPESurf@@QAA@HHPAXHW4EGPEFormat@@@Z 10004ef4 f i surf.obj
 0001:00003f48       ??_EGPESurf@@UAAPAXI@Z     10004f48 f i surf.obj
 0001:00003f48       ??_GGPESurf@@UAAPAXI@Z     10004f48 f i surf.obj
 0001:00003f6c       ?SetVisibleSurface@SGX@@UAAXPAVGPESurf@@H@Z 10004f6c f   surf.obj
 0001:00003f70       ??0SGXSurf@@QAA@HHHW4EGPEFormat@@PAU_PVR2DMEMINFO@@PAXPAPAU2@@Z 10004f70 f   surf.obj
 0001:00003fd8       ??1SGXSurf@@UAA@XZ         10004fd8 f   surf.obj
 0001:00004038       ?AllocSurface@SGX@@UAAJPAPAVGPESurf@@HHW4EGPEFormat@@H@Z 10005038 f   surf.obj
 0001:000041e8       ?GetPrimarySurface@SGX@@AAAPAVSGXSurf@@HHHW4EGPEFormat@@@Z 100051e8 f   surf.obj
 0001:00004288       ??_GSGXSurf@@UAAPAXI@Z     10005288 f i surf.obj
 0001:00004288       ??_ESGXSurf@@UAAPAXI@Z     10005288 f i surf.obj
 0001:000042ac       DllMain                    100052ac f   gpe:ddi_if.obj
 0001:000042e8       ?SafeGetGPE@@YAPAVGPE@@PAX@Z 100052e8 f   gpe:ddi_if.obj
 0001:00004354       ?SetSurfaceFormat@@YAXPAVGPESurf@@PAU_XLATEOBJ@@K@Z 10005354 f   gpe:ddi_if.obj
 0001:000044e0       DrvContrastControl         100054e0 f   gpe:ddi_if.obj
 0001:00004504       DrvPowerHandler            10005504 f   gpe:ddi_if.obj
 0001:0000452c       DrvEscape                  1000552c f   gpe:ddi_if.obj
 0001:00004674       DrvDisableDriver           10005674 f   gpe:ddi_if.obj
 0001:000046a4       DrvDisablePDEV             100056a4 f   gpe:ddi_if.obj
 0001:000046d0       DrvDisableSurface          100056d0 f   gpe:ddi_if.obj
 0001:000046f4       DrvEnableSurface           100056f4 f   gpe:ddi_if.obj
 0001:00004738       DrvCreateDeviceBitmap      10005738 f   gpe:ddi_if.obj
 0001:000047d4       DrvDeleteDeviceBitmap      100057d4 f   gpe:ddi_if.obj
 0001:00004814       DrvMovePointer             10005814 f   gpe:ddi_if.obj
 0001:00004834       DrvSetPointerShape         10005834 f   gpe:ddi_if.obj
 0001:00004948       DrvSetPalette              10005948 f   gpe:ddi_if.obj
 0001:000049d4       DrvFillPath                100059d4 f   gpe:ddi_if.obj
 0001:00004d90       DrvRealizeBrush            10005d90 f   gpe:ddi_if.obj
 0001:00005008       DrvGetModes                10006008 f   gpe:ddi_if.obj
 0001:0000510c       DrvEnablePDEV              1000610c f   gpe:ddi_if.obj
 0001:0000543c       DrvCopyBits                1000643c f   gpe:ddi_if.obj
 0001:0000544c       ?ClipBlt@@YAJPAVGPE@@PAUGPEBltParms@@@Z 1000644c f   gpe:ddi_if.obj
 0001:000056b0       ?AAGetMaskBits@@YAXPAK00@Z 100066b0 f   gpe:ddi_if.obj
 0001:000056f0       ?GPEEnableDriver@@YAHKKPAUtagDrvEnableData@@PAU_ENGCALLBACKS@@@Z 100066f0 f   gpe:ddi_if.obj
 0001:00005824       AnyBlt                     10006824 f   gpe:ddi_if.obj
 0001:00006044       DrvAnyBlt                  10007044 f   gpe:ddi_if.obj
 0001:000060b8       DrvTransparentBlt          100070b8 f   gpe:ddi_if.obj
 0001:00006138       DrvBitBlt                  10007138 f   gpe:ddi_if.obj
 0001:0000621c       DrvPaint                   1000721c f   gpe:ddi_if.obj
 0001:0000628c       ?EmulatedBlt_Internal@GPE@@QAAJPAUGPEBltParms@@@Z 1000728c f   gpe:swblt.obj
 0001:000084a4       ?EmulatedBlt_Bilinear@GPE@@QAAJPAUGPEBltParms@@@Z 100094a4 f   gpe:swblt.obj
 0001:00008d34       ?EmulatedBlt_Halftone@GPE@@QAAJPAUGPEBltParms@@@Z 10009d34 f   gpe:swblt.obj
 0001:000095d8       ?EmulatedBltRotate_Internal@GPE@@QAAJPAUGPEBltParms@@@Z 1000a5d8 f   gpe:swblt.obj
 0001:0000c2b0       ?EmulatedBltRotate_Bilinear@GPE@@QAAJPAUGPEBltParms@@@Z 1000d2b0 f   gpe:swblt.obj
 0001:0000d16c       ?EmulatedBltRotate_Halftone@GPE@@QAAJPAUGPEBltParms@@@Z 1000e16c f   gpe:swblt.obj
 0001:0000de5c       ?SelectBlt@GPE@@IAAJPAUGPEBltParms@@P81@AAJ0@Z@Z 1000ee5c f   gpe:swblt.obj
 0001:0000e244       ?EmulatedBlt@GPE@@QAAJPAUGPEBltParms@@@Z 1000f244 f   gpe:swblt.obj
 0001:0000e25c       ??0GPE@@QAA@XZ             1000f25c f   gpe:gpe.obj
 0001:0000e2a4       ??1GPE@@UAA@XZ             1000f2a4 f   gpe:gpe.obj
 0001:0000e2b4       ?ContrastControl@GPE@@UAAHKPAK@Z 1000f2b4 f   gpe:gpe.obj
 0001:0000e2bc       ?PowerHandler@GPE@@UAAXH@Z 1000f2bc f   gpe:gpe.obj
 0001:0000e2c0       ?GetPalette@GPE@@UAAJPAPAUtagPALETTEENTRY@@PAG@Z 1000f2c0 f   gpe:gpe.obj
 0001:0000e308       ?DrvEscape@GPE@@UAAKPAU_SURFOBJ@@KKPAXK1@Z 1000f308 f   gpe:gpe.obj
 0001:0000e310       ?GetGraphicsCaps@GPE@@UAAKXZ 1000f310 f   gpe:gpe.obj
 0001:0000e318       ?GetPhysicalVideoMemory@GPE@@UAAXPAK0@Z 1000f318 f   gpe:gpe.obj
 0001:0000e31c       ?SetVisibleSurface@GPE@@UAAXPAVGPESurf@@@Z 1000f31c f   gpe:gpe.obj
 0001:0000e320       ?FlipInProgress@GPE@@UAAHXZ 1000f320 f   gpe:gpe.obj
 0001:0000e328       ?WaitForVBlank@GPE@@UAAXXZ 1000f328 f   gpe:gpe.obj
 0001:0000e32c       ?SurfaceBusyFlipping@GPE@@UAAHPAVGPESurf@@@Z 1000f32c f   gpe:gpe.obj
 0001:0000e334       ?IsBusy@GPE@@UAAHXZ        1000f334 f   gpe:gpe.obj
 0001:0000e33c       ?WaitForNotBusy@GPE@@UAAXXZ 1000f33c f   gpe:gpe.obj
 0001:0000e340       ?AvailableVideoMemory@GPE@@UAAKXZ 1000f340 f   gpe:gpe.obj
 0001:0000e348       ?ScanLine@GPE@@UAAHXZ      1000f348 f   gpe:gpe.obj
 0001:0000e350       ?ProcessCommandBlock@GPE@@UAAJPAE@Z 1000f350 f   gpe:gpe.obj
 0001:0000e35c       ?GetScreenDimensions@GPE@@UAAHPAUGPEScreenProps@@@Z 1000f35c f   gpe:gpe.obj
 0001:0000e5a4       ?IsPaletteSettable@GPE@@UAAHXZ 1000f5a4 f   gpe:gpe.obj
 0001:0000e5bc       ?RotateRectl@GPE@@QAAXPAU_RECTL@@@Z 1000f5bc f   gpe:gpe.obj
 0001:0000e66c       ?GetClearTypeRGBMasks@GPE@@UAAPAKXZ 1000f66c f   gpe:gpe.obj
 0001:0000e67c       ?DisablePrimary@GPE@@UAAHXZ 1000f67c f   gpe:gpe.obj
 0001:0000e6b8       ?Init@GPESurf@@QAAXHHPAXHW4EGPEFormat@@@Z 1000f6b8 f   gpe:gpe.obj
 0001:0000e710       ?RotateLineParms@GPESurf@@QAAXPAUGPELineParms@@@Z 1000f710 f   gpe:gpe.obj
 0001:0000e7dc       ?SetRotation@GPESurf@@QAAXHHH@Z 1000f7dc f   gpe:gpe.obj
 0001:0000e804       ?RotateRectl@GPESurf@@QAAXPAU_RECTL@@@Z 1000f804 f   gpe:gpe.obj
 0001:0000e8b4       ?RotateRectlBack@GPESurf@@QAAXPAU_RECTL@@@Z 1000f8b4 f   gpe:gpe.obj
 0001:0000e96c       ?GetPtr@GPESurf@@QAAPAEHH@Z 1000f96c f   gpe:gpe.obj
 0001:0000ea48       ??1GPEFormat@@QAA@XZ       1000fa48 f   gpe:gpe.obj
 0001:0000ea7c       ??_EGPE@@UAAPAXI@Z         1000fa7c f i gpe:gpe.obj
 0001:0000ea7c       ??_GGPE@@UAAPAXI@Z         1000fa7c f i gpe:gpe.obj
 0001:0000eaa4       ??0GPESurf@@QAA@HHW4EGPEFormat@@@Z 1000faa4 f   gpe:gpe.obj
 0001:0000eb94       ??1GPESurf@@UAA@XZ         1000fb94 f   gpe:gpe.obj
 0001:0000ebd0       ?EmulatedLine@GPE@@QAAJPAUGPELineParms@@@Z 1000fbd0 f   gpe:swline.obj
 0001:0000f31c       ?vClearTypeLookupTableLoop@@YAXKPAU_BLENDINFO@@KK@Z 1001031c f   gpe:rctblt.obj
 0001:0000f6f0       ?pvFillOpaqTableCT@@YAPAXKKKPAU_BLENDINFO@@@Z 100106f0 f   gpe:rctblt.obj
 0001:0000f76c       ?ulBlendPixelCT@@YAKPAU_BLENDINFO@@KPAU_F_RGB@@@Z 1001076c f   gpe:rctblt.obj
 0001:0000f8a8       ?ulBlendPixelCT8bpp@@YAKPAU_BLENDINFO@@KPAU_F_RGB@@@Z 100108a8 f   gpe:rctblt.obj
 0001:0000f984       ?ClearTypeBltDst16@ClearTypeBlt@@QAAJPAUGPEBltParms@@@Z 10010984 f   gpe:rctblt.obj
 0001:0000fb60       ?ClearTypeBltDst24@ClearTypeBlt@@QAAJPAUGPEBltParms@@@Z 10010b60 f   gpe:rctblt.obj
 0001:0000fd54       ?ClearTypeBltDst32@ClearTypeBlt@@QAAJPAUGPEBltParms@@@Z 10010d54 f   gpe:rctblt.obj
 0001:0000ff1c       ?ClearTypeBltDst8@ClearTypeBlt@@QAAJPAUGPEBltParms@@@Z 10010f1c f   gpe:rctblt.obj
 0001:000100e8       ?SetClearTypeBltMasks@@YAXKKK@Z 100110e8 f   gpe:rctblt.obj
 0001:000101c4       ?SetClearTypeBltPalette@@YAXPAUtagPALETTEENTRY@@H@Z 100111c4 f   gpe:rctblt.obj
 0001:000101d4       ?SetClearTypeBltGamma@@YAXK@Z 100111d4 f   gpe:rctblt.obj
 0001:00010394       ?GetGammaValue@@YAHPAK@Z   10011394 f   gpe:rctblt.obj
 0001:000103b0       ?SetGammaValue@@YAHKH@Z    100113b0 f   gpe:rctblt.obj
 0001:0001046c       ?ClearTypeBltInit@@YAHPAUGPEMode@@PAKPAUtagPALETTEENTRY@@I@Z 1001146c f   gpe:rctblt.obj
 0001:000105bc       ?ClearTypeBltSelect@@YAJPAUGPEBltParms@@@Z 100115bc f   gpe:rctblt.obj
 0001:00010658       ?Init@LRU@@QAAHG@Z         10011658 f   gpe:swconvrt.obj
 0001:00010724       ?Find@LRU@@QAAFK@Z         10011724 f   gpe:swconvrt.obj
 0001:000107fc       ?Add@LRU@@QAAFK@Z          100117fc f   gpe:swconvrt.obj
 0001:0001085c       ?Free@LRU@@QAAXXZ          1001185c f   gpe:swconvrt.obj
 0001:000108b8       ?InitMaskInfo@MaskInfo@@QAAXPAU_XLATEOBJ@@KG@Z 100118b8 f   gpe:swconvrt.obj
 0001:0001098c       ?Init@MaskColorConverter@@QAAXPAU_XLATEOBJ@@@Z 1001198c f   gpe:swconvrt.obj
 0001:000109c0       ?Init@GroupColorConverter@@QAAXPAU_XLATEOBJ@@@Z 100119c0 f   gpe:swconvrt.obj
 0001:00010bf4       ?RGBToFromBGR@MaskColorConverter@@QAAKK@Z 10011bf4 f   gpe:swconvrt.obj
 0001:00010c2c       ?MaskedSrcToRGB@MaskColorConverter@@QAAKK@Z 10011c2c f   gpe:swconvrt.obj
 0001:00010c9c       ?MaskedSrcToRGB@GroupColorConverter@@QAAKK@Z 10011c9c f   gpe:swconvrt.obj
 0001:00010d0c       ?MaskedSrcToBGR@MaskColorConverter@@QAAKK@Z 10011d0c f   gpe:swconvrt.obj
 0001:00010d7c       ?RGBSrcToMaskedDst@MaskColorConverter@@QAAKK@Z 10011d7c f   gpe:swconvrt.obj
 0001:00010dc0       ?BGRSrcToMaskedDst@MaskColorConverter@@QAAKK@Z 10011dc0 f   gpe:swconvrt.obj
 0001:00010e04       ?MaskedSrcToMaskedDst@MaskColorConverter@@QAAKK@Z 10011e04 f   gpe:swconvrt.obj
 0001:00010e84       ?AnyToMono@MonoColorConverter@@QAAKK@Z 10011e84 f   gpe:swconvrt.obj
 0001:00010e98       DrvRealizeColor            10011e98 f   gpe:swconvrt.obj
 0001:0001100c       DrvUnrealizeColor          1001200c f   gpe:swconvrt.obj
 0001:00011118       ?Init@LookupColorConverter@@QAAXPAU_XLATEOBJ@@@Z 10012118 f   gpe:swconvrt.obj
 0001:000112fc       ?MaskedSrcToPaletteDst@GroupColorConverter@@QAAKK@Z 100122fc f   gpe:swconvrt.obj
 0001:000114ac       ?AllocConverters@@YAHXZ    100124ac f   gpe:swconvrt.obj
 0001:0001155c       ?FreeConverters@@YAXXZ     1001255c f   gpe:swconvrt.obj
 0001:000115bc       ?InitConverter@ColorConverter@@SAXPAU_XLATEOBJ@@PAPAV1@PAP81@AAKK@ZPAPAK@Z 100125bc f   gpe:swconvrt.obj
 0001:0001180c       ?SafeCallLine@@YAJPAVGPE@@PAUGPELineParms@@@Z 1001280c f   gpe:drvstrok.obj
 0001:0001185c       DrvStrokePath              1001285c f   gpe:drvstrok.obj
 0001:000121a0       ?AATextBltInit@@YAHP6AXPAK00@Z@Z 100131a0 f   gpe:aablt.obj
 0001:000121b8       ?AATextBltDst8@AATextBlt@@QAAJPAUGPEBltParms@@@Z 100131b8 f   gpe:aablt.obj
 0001:00012364       ?SetGamma@AAMASKINFO@@QAAXM@Z 10013364 f i gpe:aablt.obj
 0001:00012564       ?BlendPixelAA@AAMASKINFO@@QAAKKE@Z 10013564 f   gpe:aablt.obj
 0001:000128d0       ?SetAAGammaValue@@YAHKH@Z  100138d0 f   gpe:aablt.obj
 0001:000129f0       ?AATextBltDst16@AATextBlt@@QAAJPAUGPEBltParms@@@Z 100139f0 f   gpe:aablt.obj
 0001:00012c20       ?AATextBltDst24@AATextBlt@@QAAJPAUGPEBltParms@@@Z 10013c20 f   gpe:aablt.obj
 0001:00012e70       ?AATextBltDst32@AATextBlt@@QAAJPAUGPEBltParms@@@Z 10013e70 f   gpe:aablt.obj
 0001:00013098       ?AATextBltSelect@@YAJPAUGPEBltParms@@@Z 10014098 f   gpe:aablt.obj
 0001:0001314c       ??0TmpGPESurf@@QAA@PAU_SURFOBJ@@0PAV0@@Z 1001414c f   gpe:TmpGPESurf.obj
 0001:00013204       ??0EdgeList@@QAA@H@Z       10014204 f   gpe:swfill.obj
 0001:0001324c       ??1EdgeList@@QAA@XZ        1001424c f   gpe:swfill.obj
 0001:00013268       ?AddEdge@EdgeList@@QAAJJJJJ@Z 10014268 f   gpe:swfill.obj
 0001:0001349c       ?Fill@EdgeList@@QAAJPAUGPEBltParms@@PAU_RECTL@@PAVGPE@@@Z 1001449c f   gpe:swfill.obj
 0001:0001393c       ?drvRectFill32@@YAXPAVGPESurf@@PAU_DRVGRADIENTRECTDATA@@@Z 1001493c f   gpe:rdrvgradfill.obj
 0001:0001407c       ?drvRectFill24@@YAXPAVGPESurf@@PAU_DRVGRADIENTRECTDATA@@@Z 1001507c f   gpe:rdrvgradfill.obj
 0001:000146bc       ?drvRectFill16@@YAXPAVGPESurf@@PAU_DRVGRADIENTRECTDATA@@H@Z 100156bc f   gpe:rdrvgradfill.obj
 0001:00014bb4       ?drvRectFill16_565@@YAXPAVGPESurf@@PAU_DRVGRADIENTRECTDATA@@@Z 10015bb4 f   gpe:rdrvgradfill.obj
 0001:00014bc8       ?drvRectFill16_555@@YAXPAVGPESurf@@PAU_DRVGRADIENTRECTDATA@@@Z 10015bc8 f   gpe:rdrvgradfill.obj
 0001:00014c20       ?drvRectFill16Bitfields@@YAXPAVGPESurf@@PAU_DRVGRADIENTRECTDATA@@@Z 10015c20 f   gpe:rdrvgradfill.obj
 0001:00014c34       ?drvRectFillPalIndex@@YAXPAVGPESurf@@PAU_DRVGRADIENTRECTDATA@@H@Z 10015c34 f   gpe:rdrvgradfill.obj
 0001:0001510c       ?drvRectFill8@@YAXPAVGPESurf@@PAU_DRVGRADIENTRECTDATA@@@Z 1001610c f   gpe:rdrvgradfill.obj
 0001:00015120       ?drvRectFill4@@YAXPAVGPESurf@@PAU_DRVGRADIENTRECTDATA@@@Z 10016120 f   gpe:rdrvgradfill.obj
 0001:00015134       ?drvRectFill1@@YAXPAVGPESurf@@PAU_DRVGRADIENTRECTDATA@@@Z 10016134 f   gpe:rdrvgradfill.obj
 0001:0001582c       DrvGradientFill            1001682c f   gpe:rdrvgradfill.obj
 0001:00016094       DrvAlphaBlend              10017094 f   gpe:drvalphablend.obj
 0001:0001611c       GenBltInitialize           1001711c f   gpe:genblt.obj
 0001:000162d4       ?ClockOverflow@@YAXXZ      100172d4 f   gpe:genblt.obj
 0001:00016314       ?FunctionCacheLookup@@YAPAUGenBltFunction@@PAUGenBltSignature@@@Z 10017314 f   gpe:genblt.obj
 0001:00016380       ?GetFnCacheMem@@YAPAUGenBltFunction@@PAUGenBltSignature@@@Z 10017380 f   gpe:genblt.obj
 0001:00016400       ?GetBltFunction@@YAPAUGenBltFunction@@PAUGenBltSignature@@@Z 10017400 f   gpe:genblt.obj
 0001:000164b4       ?GPEFormatToGenBltFormat@@YA?AW4GenBltFormat@@PAVGPEFormat@@W4EGPEFormat@@@Z 100174b4 f   gpe:genblt.obj
 0001:0001662c       GenBltSetMode              1001762c f   gpe:genblt.obj
 0001:00016838       ?GenerateSignature@@YAHPAUGPEBltParms@@PAUGenBltSignature@@@Z 10017838 f   gpe:genblt.obj
 0001:00016cc4       ?ProcessROP3@@YAKKKKEE@Z   10017cc4 f   gpe:BltHelpers.obj
 0001:00016d84       ?RGBError@@YAKKK@Z         10017d84 f   gpe:BltHelpers.obj
 0001:00016dc8       ?FillMasksAndShifts@@YAXPAVGPESurf@@PAK1@Z 10017dc8 f   gpe:BltHelpers.obj
 0001:00016e38       ?ClipRect@@YA_NPAU_RECTL@@PBU1@1@Z 10017e38 f   gpe:BltHelpers.obj
 0001:00016eb8       ?AveragePixels@@YAKKKHHPAK0@Z 10017eb8 f   gpe:BltHelpers.obj
 0001:00017018       ?AverageAndClampPixels@@YAKKKHHPAK0@Z 10018018 f   gpe:BltHelpers.obj
 0001:000171bc       ?HalftoneBlend16Bpp@@YAXPAEKHHPAK1@Z 100181bc f   gpe:BltHelpers.obj
 0001:000171f4       ?HalftoneBlend24Bpp@@YAXPAEKHHPAK1@Z 100181f4 f   gpe:BltHelpers.obj
 0001:00017248       ?HalftoneBlend32Bpp@@YAXPAEKHHPAK1@Z 10018248 f   gpe:BltHelpers.obj
 0001:0001727c       ?InitPixelIterator@PixelIterator@@QAAXPAVGPESurf@@HHPAU_RECTL@@HH@Z 1001827c f   gpe:PixelIterator.obj
 0001:0001744c       ?InitPixelIterator@PixelIteratorRotate@@QAAXPAVGPESurf@@HHPAU_RECTL@@HH@Z 1001844c f   gpe:PixelIterator.obj
 0001:000175ac       ?GetPtr@PixelIteratorRotate@@QAAPAEXZ 100185ac f   gpe:PixelIterator.obj
 0001:00017698       ?InitBrushPixelIterator@BrushPixelIterator@@QAAXPAVGPESurf@@HHPAU_RECTL@@@Z 10018698 f   gpe:PixelIterator.obj
 0001:00017784       ?WrappedGeneratedBlt@GPE@@QAAJPAUGPEBltParms@@@Z 10018784 f   gpe:GenBltGpe.obj
 0001:00017884       GeneratedBltSelect         10018884 f   gpe:GenBltGpe.obj
 0001:000178d4       EmulatedBltSelect02        100188d4 f   gpe:ebbltsel.obj
 0001:000178dc       EmulatedBltSelect08        100188dc f   gpe:ebbltsel.obj
 0001:00017b04       EmulatedBltSelect16        10018b04 f   gpe:ebbltsel.obj
 0001:00017cd8       ?IsSurface_R5_G6_B5@@YAHPAVGPESurf@@@Z 10018cd8 f i gpe:FastBlt.obj
 0001:00017d30       ?IsSurface_A8_R8_G8_B8@@YAHPAVGPESurf@@@Z 10018d30 f i gpe:FastBlt.obj
 0001:00017d94       ?CanUse_Blt_Stretch_Alpha_32To16at565@@YAHPAUGPEBltParms@@@Z 10018d94 f i gpe:FastBlt.obj
 0001:00017e90       ?Blt_Stretch_Alpha_32To16at565@Emulator@@QAAJPAUGPEBltParms@@@Z 10018e90 f   gpe:FastBlt.obj
 0001:0001862c       ?CanUse_Blt_NoStretch_Alpha_32To16at565@@YAHPAUGPEBltParms@@@Z 1001962c f i gpe:FastBlt.obj
 0001:00018668       ?Blt_NoStretch_Alpha_32To16at565@Emulator@@QAAJPAUGPEBltParms@@@Z 10019668 f   gpe:FastBlt.obj
 0001:000189b4       ?CanUse_Blt_NoStretch_Alpha_24To24@@YAHPAUGPEBltParms@@@Z 100199b4 f i gpe:FastBlt.obj
 0001:00018a4c       ?Blt_NoStretch_Alpha_24To24_Aligned@@YAJPAKH0HHHK@Z 10019a4c f   gpe:FastBlt.obj
 0001:00018b90       ?Blt_NoStretch_Alpha_24To24@Emulator@@QAAJPAUGPEBltParms@@@Z 10019b90 f   gpe:FastBlt.obj
 0001:00018d68       ?CanUse_Blt_NoStretch_Alpha_16To16@@YAHPAUGPEBltParms@@@Z 10019d68 f i gpe:FastBlt.obj
 0001:00018e10       ?Blt_NoStretch_Alpha_16To16@Emulator@@QAAJPAUGPEBltParms@@@Z 10019e10 f   gpe:FastBlt.obj
 0001:00018fec       ?CanUse_Blt_NoStretch_Trans_16To16@@YAHPAUGPEBltParms@@@Z 10019fec f i gpe:FastBlt.obj
 0001:00019088       ?Blt_NoStretch_Trans_16To16@Emulator@@QAAJPAUGPEBltParms@@@Z 1001a088 f   gpe:FastBlt.obj
 0001:00019150       ?CanUse_Blt_Stretch_Trans_16To16@@YAHPAUGPEBltParms@@@Z 1001a150 f i gpe:FastBlt.obj
 0001:000191f0       ?CanUse_Blt_NoStretch_NoTrans_32To16at565@@YAHPAUGPEBltParms@@@Z 1001a1f0 f i gpe:FastBlt.obj
 0001:00019288       ?Blt_NoStretch_NoTrans_32To16at565@Emulator@@QAAJPAUGPEBltParms@@@Z 1001a288 f   gpe:FastBlt.obj
 0001:00019354       ?CanUse_Blt_NoStretch_NoTrans_16at565To32@@YAHPAUGPEBltParms@@@Z 1001a354 f i gpe:FastBlt.obj
 0001:000193f8       ?Blt_NoStretch_NoTrans_16at565To32@Emulator@@QAAJPAUGPEBltParms@@@Z 1001a3f8 f   gpe:FastBlt.obj
 0001:000194c0       ?CanUse_Blt_NoStretch_NoTrans_24To24@@YAHPAUGPEBltParms@@@Z 1001a4c0 f i gpe:FastBlt.obj
 0001:00019558       ?Blt_NoStretch_NoTrans_24To24@Emulator@@QAAJPAUGPEBltParms@@@Z 1001a558 f   gpe:FastBlt.obj
 0001:00019610       ?CanUse_Blt_NoStretch_NoTrans_16To16@@YAHPAUGPEBltParms@@@Z 1001a610 f i gpe:FastBlt.obj
 0001:000196a8       ?Blt_NoStretch_NoTrans_16To16@Emulator@@QAAJPAUGPEBltParms@@@Z 1001a6a8 f   gpe:FastBlt.obj
 0001:0001975c       ?CanUse_Blt_Text_32@@YAHPAUGPEBltParms@@@Z 1001a75c f i gpe:FastBlt.obj
 0001:000197e8       ?Blt_Text_32@Emulator@@QAAJPAUGPEBltParms@@@Z 1001a7e8 f   gpe:FastBlt.obj
 0001:000198e0       ?CanUse_Blt_Fill_32@@YAHPAUGPEBltParms@@@Z 1001a8e0 f i gpe:FastBlt.obj
 0001:0001993c       ?Blt_Fill_32@Emulator@@QAAJPAUGPEBltParms@@@Z 1001a93c f   gpe:FastBlt.obj
 0001:000199d4       ?CanUse_Blt_Fill_24@@YAHPAUGPEBltParms@@@Z 1001a9d4 f i gpe:FastBlt.obj
 0001:00019a30       ?Blt_Fill_24@Emulator@@QAAJPAUGPEBltParms@@@Z 1001aa30 f   gpe:FastBlt.obj
 0001:00019ae8       ?Blt_Stretch_Trans_16To16@Emulator@@QAAJPAUGPEBltParms@@@Z 1001aae8 f   gpe:FastBlt.obj
 0001:0001a188       FastBltSelect              1001b188 f   gpe:FastBlt.obj
 0001:0001a374       GenBltCpuInitialize        1001b374 f   gpe:genblt_arm.obj
 0001:0001a3a0       ?RopRecurse@@YAFPAKF@Z     1001b3a0 f   gpe:parse.obj
 0001:0001a4c0       ?ConvertRecurse@@YAFPAKKF@Z 1001b4c0 f   gpe:parse.obj
 0001:0001a6b8       ?GenBltInvariantParser@@YA_NPAK0PAUGenBltSignature@@@Z 1001b6b8 f   gpe:parse.obj
 0001:0001a9a4       ?InvariantRecurse@@YAFPAKKKHF@Z 1001b9a4 f   gpe:parse.obj
 0001:0001acec       ?InvariantInitialize@@YAHPAK@Z 1001bcec f   gpe:parse.obj
 0001:0001af28       ?BRegFromBltSig@@YAKPAUGenBltSignature@@@Z 1001bf28 f   gpe:InitRegs.obj
 0001:0001b07c       ?InitPCodeRegs@@YAXPAUGPEBltParms@@PAUPCodeRegisters_t@@@Z 1001c07c f   gpe:InitRegs.obj
 0001:0001bdf0       ?EmulatedBltSrcCopy0108@Emulator@@QAAJPAUGPEBltParms@@@Z 1001cdf0 f   gpe:ebcp0108.obj
 0001:0001c264       ?EmulatedBltSrcCopy0408@Emulator@@QAAJPAUGPEBltParms@@@Z 1001d264 f   gpe:ebcp0408.obj
 0001:0001c3f0       ?EmulatedBltSrcCopy0808@Emulator@@QAAJPAUGPEBltParms@@@Z 1001d3f0 f   gpe:ebcopy08.obj
 0001:0001c770       ?EmulatedBltSrcPaint0808@Emulator@@QAAJPAUGPEBltParms@@@Z 1001d770 f   gpe:ebspnt08.obj
 0001:0001cb70       ?EmulatedBltPatternCopy08@Emulator@@QAAJPAUGPEBltParms@@@Z 1001db70 f   gpe:ebpcpy08.obj
 0001:0001cf4c       ?EmulatedBltAlphaText08@Emulator@@QAAJPAUGPEBltParms@@@Z 1001df4c f   gpe:ebalph08.obj
 0001:0001cf6c       ?EmulatedBltText08@Emulator@@QAAJPAUGPEBltParms@@@Z 1001df6c f   gpe:ebtext08.obj
 0001:0001d0c4       ?EmulatedBltFill08@Emulator@@QAAJPAUGPEBltParms@@@Z 1001e0c4 f   gpe:ebfill08.obj
 0001:0001d158       ?EmulatedBltDstInvert08@Emulator@@QAAJPAUGPEBltParms@@@Z 1001e158 f   gpe:ebdinv08.obj
 0001:0001d260       ?EmulatedBltPatInvert08@Emulator@@QAAJPAUGPEBltParms@@@Z 1001e260 f   gpe:ebpinv08.obj
 0001:0001d388       ?EmulatedBltPatternInvert08@Emulator@@QAAJPAUGPEBltParms@@@Z 1001e388 f   gpe:ebp08.obj
 0001:0001d5ec       ?EmulatedBltSrcInvert0808@Emulator@@QAAJPAUGPEBltParms@@@Z 1001e5ec f   gpe:ebsinv08.obj
 0001:0001d9ec       ?EmulatedBltSrcAnd0808@Emulator@@QAAJPAUGPEBltParms@@@Z 1001e9ec f   gpe:ebsand08.obj
 0001:0001ddec       ?EmulatedBltSrcPaint1616@Emulator@@QAAJPAUGPEBltParms@@@Z 1001edec f   gpe:EBSPNT16.obj
 0001:0001e1ec       ?EmulatedBltSrcCopy0116@Emulator@@QAAJPAUGPEBltParms@@@Z 1001f1ec f   gpe:ebcp0116.obj
 0001:0001e664       ?EmulatedBltSrcCopy0416@Emulator@@QAAJPAUGPEBltParms@@@Z 1001f664 f   gpe:ebcp0416.obj
 0001:0001e7f4       ?EmulatedBltSrcCopy1616@Emulator@@QAAJPAUGPEBltParms@@@Z 1001f7f4 f   gpe:EBCOPY16.obj
 0001:0001eb9c       ?EmulatedBltFill16@Emulator@@QAAJPAUGPEBltParms@@@Z 1001fb9c f   gpe:ebfill16.obj
 0001:0001ec5c       ?EmulatedBltSrcInvert1616@Emulator@@QAAJPAUGPEBltParms@@@Z 1001fc5c f   gpe:EBSINV16.obj
 0001:0001f05c       ?EmulatedBltSrcAnd1616@Emulator@@QAAJPAUGPEBltParms@@@Z 1002005c f   gpe:ebsand16.obj
 0001:0001f45c       ?EmulatedBltAlphaText16@Emulator@@QAAJPAUGPEBltParms@@@Z 1002045c f   gpe:ebalph16.obj
 0001:0001f47c       ?EmulatedBltText16@Emulator@@QAAJPAUGPEBltParms@@@Z 1002047c f   gpe:ebtext16.obj
 0001:0001f5d4       OutputDebugStringW         100205d4 f   coredll:COREDLL.dll
 0001:0001f5e4       NKDbgPrintfW               100205e4 f   coredll:COREDLL.dll
 0001:0001f5f4       SetLastError               100205f4 f   coredll:COREDLL.dll
 0001:0001f604       RegCloseKey                10020604 f   coredll:COREDLL.dll
 0001:0001f614       RegQueryValueExW           10020614 f   coredll:COREDLL.dll
 0001:0001f624       RegOpenKeyExW              10020624 f   coredll:COREDLL.dll
 0001:0001f634       AdvertiseInterface         10020634 f   coredll:COREDLL.dll
 0001:0001f644       GetModuleFileNameW         10020644 f   coredll:COREDLL.dll
 0001:0001f654       DisableThreadLibraryCalls  10020654 f   coredll:COREDLL.dll
 0001:0001f664       RegSetValueExW             10020664 f   coredll:COREDLL.dll
 0001:0001f674       RegCreateKeyExW            10020674 f   coredll:COREDLL.dll
 0001:0001f684       LocalAlloc                 10020684 f   coredll:COREDLL.dll
 0001:0001f694       LocalFree                  10020694 f   coredll:COREDLL.dll
 0001:0001f6a4       LocalReAlloc               100206a4 f   coredll:COREDLL.dll
 0001:0001f6b4       VirtualFree                100206b4 f   coredll:COREDLL.dll
 0001:0001f6c4       CeSetExtendedPdata         100206c4 f   coredll:COREDLL.dll
 0001:0001f6d4       VirtualAlloc               100206d4 f   coredll:COREDLL.dll
 0001:0001f6e4       CacheRangeFlush            100206e4 f   coredll:COREDLL.dll
 0001:0001f6f4       GetPvrSrvPixelFormat       100206f4 f   libpvr2d:pvr2dblt.obj
 0001:0001f764       PVR2DQueryBlitsComplete    10020764 f   libpvr2d:pvr2dblt.obj
 0001:00020080       PVR2DBltClipped            10021080 f   libpvr2d:pvr2dblt.obj
 0001:00020084       PVR2DGetFrameBuffer        10021084 f   libpvr2d:pvr2dmode.obj
 0001:000200c0       PVR2DGetScreenMode         100210c0 f   libpvr2d:pvr2dmode.obj
 0001:000201a4       PVR2DEnumerateDevices      100211a4 f   libpvr2d:pvr2dinit.obj
 0001:00020574       PVR2DCreateDeviceContext   10021574 f   libpvr2d:pvr2dinit.obj
 0001:0002079c       PVR2DDestroyDeviceContext  1002179c f   libpvr2d:pvr2dinit.obj
 0001:000208a0       PVR2DMemAlloc              100218a0 f   libpvr2d:pvr2dmem.obj
 0001:0002095c       PVR2DMemFree               1002195c f   libpvr2d:pvr2dmem.obj
 0001:00020a20       DestroyFlipChain           10021a20 f   libpvr2d:pvr2dflip.obj
 0001:00020af8       PVRSRVEventObjectOpen      10021af8 f   srvclkm:srvclient_wince.obj
 0001:00020b60       PVRSRVEventObjectClose     10021b60 f   srvclkm:srvclient_wince.obj
 0001:00020b68       PVRSRVEventObjectWait      10021b68 f   srvclkm:srvclient_wince.obj
 0001:00020ba8       PVRSRVUnlockResource       10021ba8 f   srvclkm:srvclient_wince.obj
 0001:00020bdc       PVRSRVCallocUserModeMem    10021bdc f   srvclkm:srvclient_wince.obj
 0001:00020be8       PVRSRVClockus              10021be8 f   srvclkm:srvclient_wince.obj
 0001:00020c00       PVRSRVWaitus               10021c00 f   srvclkm:srvclient_wince.obj
 0001:00020c40       PVRSRVMemCopy              10021c40 f   srvclkm:srvclient_wince.obj
 0001:00020c44       PVRSRVMemSet               10021c44 f   srvclkm:srvclient_wince.obj
 0001:00020c48       PVRSRVCreateMutex          10021c48 f   srvclkm:srvclient_wince.obj
 0001:00020c70       PVRSRVDestroyMutex         10021c70 f   srvclkm:srvclient_wince.obj
 0001:00020c80       PVRSRVUnlockMutex          10021c80 f   srvclkm:srvclient_wince.obj
 0001:00020ca0       PVRSRVLockResource         10021ca0 f   srvclkm:srvclient_wince.obj
 0001:00020d00       PVRSRVLockMutex            10021d00 f   srvclkm:srvclient_wince.obj
 0001:00020d24       SGXSubmitTransferBridge    10021d24 f   srvclkm:bridged_sgx_glue.obj
 0001:00020d9c       SGXRegisterHWTransferContext 10021d9c f   srvclkm:bridged_sgx_glue.obj
 0001:00020e30       SGXUnregisterHWTransferContext 10021e30 f   srvclkm:bridged_sgx_glue.obj
 0001:00020ea4       SGX2DQueryBlitsComplete    10021ea4 f   srvclkm:bridged_sgx_glue.obj
 0001:00025720       SGXQueueTransfer           10026720 f   srvclkm:sgxtransfer_queue.obj
 0001:00025af0       PVRSRVEnumerateDeviceClass 10026af0 f   srvclkm:bridged_pvr_glue.obj
 0001:00025bb4       PVRSRVConnect              10026bb4 f   srvclkm:bridged_pvr_glue.obj
 0001:00025be4       PVRSRVDisconnect           10026be4 f   srvclkm:bridged_pvr_glue.obj
 0001:00025bec       PVRSRVEnumerateDevices     10026bec f   srvclkm:bridged_pvr_glue.obj
 0001:00025c98       PVRSRVAcquireDeviceData    10026c98 f   srvclkm:bridged_pvr_glue.obj
 0001:00025d1c       PVRSRVCreateDeviceMemContext 10026d1c f   srvclkm:bridged_pvr_glue.obj
 0001:00025df4       PVRSRVDestroyDeviceMemContext 10026df4 f   srvclkm:bridged_pvr_glue.obj
 0001:00025e68       PVRSRVGetDeviceMemHeapInfo 10026e68 f   srvclkm:bridged_pvr_glue.obj
 0001:00025f3c       PVRSRVUnwrapExtMemory      10026f3c f   srvclkm:bridged_pvr_glue.obj
 0001:00025ff0       PVRSRVMapDeviceClassMemory 10026ff0 f   srvclkm:bridged_pvr_glue.obj
 0001:00026154       PVRSRVUnmapDeviceClassMemory 10027154 f   srvclkm:bridged_pvr_glue.obj
 0001:00026204       PVRSRVGetMiscInfo          10027204 f   srvclkm:bridged_pvr_glue.obj
 0001:000262e4       PVRSRVGetMMUContextPDDevPAddr 100272e4 f   srvclkm:bridged_pvr_glue.obj
 0001:00026340       PVRSRVUnmapDeviceMemory    10027340 f   srvclkm:bridged_pvr_glue.obj
 0001:000263d8       PVRSRVOpenDCDevice         100273d8 f   srvclkm:bridged_pvr_dc_glue.obj
 0001:00026468       PVRSRVCloseDCDevice        10027468 f   srvclkm:bridged_pvr_dc_glue.obj
 0001:000264f0       PVRSRVEnumDCFormats        100274f0 f   srvclkm:bridged_pvr_dc_glue.obj
 0001:000265bc       PVRSRVEnumDCDims           100275bc f   srvclkm:bridged_pvr_dc_glue.obj
 0001:00026698       PVRSRVGetDCSystemBuffer    10027698 f   srvclkm:bridged_pvr_dc_glue.obj
 0001:00026728       PVRSRVGetDCInfo            10027728 f   srvclkm:bridged_pvr_dc_glue.obj
 0001:000267ec       PVRSRVDestroyDCSwapChain   100277ec f   srvclkm:bridged_pvr_dc_glue.obj
 0001:0002685c       PVRSRVSwapToDCSystem       1002785c f   srvclkm:bridged_pvr_dc_glue.obj
 0001:000268d0       PVRSRVGetCurrentProcessID  100278d0 f   srvclkm:osfnex_clientkm.obj
 0001:000268d8       PVRSRVAllocUserModeMem     100278d8 f   srvclkm:osfnex_clientkm.obj
 0001:000268e4       PVRSRVFreeUserModeMem      100278e4 f   srvclkm:osfnex_clientkm.obj
 0001:000268f0       PVRSRVReleaseMiscInfo      100278f0 f   srvclkm:pvr_glue.obj
 0001:000269bc       PVRSRVAllocDeviceMem       100279bc f   srvclkm:pvr_glue.obj
 0001:00026acc       PVRSRVFreeDeviceMem        10027acc f   srvclkm:pvr_glue.obj
 0001:0002752c       SGXDestroyTransferContext  1002852c f   srvclkm:sgxtransfer_context.obj
 0001:000277a4       SGXCreateTransferContext   100287a4 f   srvclkm:sgxtransfer_context.obj
 0001:00027d28       PVRSRVBridgeCall           10028d28 f   srvclkm:pvr_bridge_clientkm.obj
 0001:00027e28       OpenServices               10028e28 f   srvclkm:pvr_bridge_clientkm.obj
 0001:00027ee0       CloseServices              10028ee0 f   srvclkm:pvr_bridge_clientkm.obj
 0001:00027f44       SGXTQ_FixedIntDiv          10028f44 f   srvclkm:sgxtransfer_utils.obj
 0001:00027f80       SGXTQ_FixedToFloat         10028f80 f   srvclkm:sgxtransfer_utils.obj
 0001:00028000       SGXTQ_FixedToF16           10029000 f   srvclkm:sgxtransfer_utils.obj
 0001:00028080       SGXTQ_GetTAGFormat         10029080 f   srvclkm:sgxtransfer_utils.obj
 0001:000282b0       SGXTQ_GetPBEFormat         100292b0 f   srvclkm:sgxtransfer_utils.obj
 0001:0002847c       SGXTQ_FilterFromEnum       1002947c f   srvclkm:sgxtransfer_utils.obj
 0001:000284ac       SGXTQ_RotationFromEnum     100294ac f   srvclkm:sgxtransfer_utils.obj
 0001:000284ec       SGXTQ_MemLayoutFromEnum    100294ec f   srvclkm:sgxtransfer_utils.obj
 0001:000285c0       SGXTQ_ShaderFromAlpha      100295c0 f   srvclkm:sgxtransfer_utils.obj
 0001:00028618       SGXTQ_ShaderFromRop        10029618 f   srvclkm:sgxtransfer_utils.obj
 0001:0002873c       SGXTQ_WriteUSEMovToReg     1002973c f   srvclkm:sgxtransfer_utils.obj
 0001:000287e4       SGXTQ_GetStrideGran        100297e4 f   srvclkm:sgxtransfer_utils.obj
 0001:00028810       SGXTQ_GetSurfaceStride     10029810 f   srvclkm:sgxtransfer_utils.obj
 0001:00028980       SGXTQ_GetSurfaceWidth      10029980 f   srvclkm:sgxtransfer_utils.obj
 0001:00028a70       SGXTQ_SetTAGState          10029a70 f   srvclkm:sgxtransfer_utils.obj
 0001:00028c04       SGXTQ_SetUSSEKick          10029c04 f   srvclkm:sgxtransfer_utils.obj
 0001:00028c54       SGXTQ_SetDMAState          10029c54 f   srvclkm:sgxtransfer_utils.obj
 0001:00028c9c       SGXTQ_SetupStridedBlit     10029c9c f   srvclkm:sgxtransfer_utils.obj
 0001:00028e8c       SGXTQ_SetPBEState          10029e8c f   srvclkm:sgxtransfer_utils.obj
 0001:00028fc4       SGXTQ_UpdateTileEvent      10029fc4 f   srvclkm:sgxtransfer_utils.obj
 0001:000290fc       SGXTQ_UpdateSecondaryPDSProgramBasic 1002a0fc f   srvclkm:sgxtransfer_utils.obj
 0001:00029174       SGXTQ_UpdateSecondaryPDSProgram1Attr 1002a174 f   srvclkm:sgxtransfer_utils.obj
 0001:0002920c       SGXTQ_UpdateSecondaryPDSProgram3Attr 1002a20c f   srvclkm:sgxtransfer_utils.obj
 0001:000292e4       SGXTQ_UpdateSecondaryPDSProgram4AttrDMA 1002a2e4 f   srvclkm:sgxtransfer_utils.obj
 0001:0002941c       SGXTQ_UpdateSecondaryPDSProgramTexSetup 1002a41c f   srvclkm:sgxtransfer_utils.obj
 0001:00029430       SGXTQ_SetupTransferRegs    1002a430 f   srvclkm:sgxtransfer_utils.obj
 0001:00029528       SGXTQ_UpdatePrimaryPDSSingleSource 1002a528 f   srvclkm:sgxtransfer_utils.obj
 0001:00029620       SGXTQ_UpdatePrimaryPDSTwoSource 1002a620 f   srvclkm:sgxtransfer_utils.obj
 0001:00029798       SGXTQ_UpdatePrimaryPDSThreeSource 1002a798 f   srvclkm:sgxtransfer_utils.obj
 0001:00029990       SGXTQ_UpdatePrimaryPDSIter 1002a990 f   srvclkm:sgxtransfer_utils.obj
 0001:00029a28       SGXTQ_UpdatePrimaryPDSKickOnly 1002aa28 f   srvclkm:sgxtransfer_utils.obj
 0001:00029aa0       SGXTQ_SetupTransferRenderBox 1002aaa0 f   srvclkm:sgxtransfer_utils.obj
 0001:00029adc       SGXTQ_SetupTransferClipRenderBox 1002aadc f   srvclkm:sgxtransfer_utils.obj
 0001:00029b4c       SGXTQ_UpdateControlObject  1002ab4c f   srvclkm:sgxtransfer_utils.obj
 0001:0002a010       SGXTQ_UpdateISPControlStream 1002b010 f   srvclkm:sgxtransfer_utils.obj
 0001:0002a3f4       SGXTQ_StagingBufferAcquireSpace 1002b3f4 f   srvclkm:sgxtransfer_utils.obj
 0001:0002a4d0       SGXTQ_GetStagingBufferDevVAddr 1002b4d0 f   srvclkm:sgxtransfer_utils.obj
 0001:0002a4e0       SGXTQ_UpdateStagingBuffer  1002b4e0 f   srvclkm:sgxtransfer_utils.obj
 0001:0002a4fc       SGXTQ_ClampInputRects      1002b4fc f   srvclkm:sgxtransfer_utils.obj
 0001:0002a57c       SGXTQ_CopyToStagingBuffer  1002b57c f   srvclkm:sgxtransfer_utils.obj
 0001:0002a5d4       SGXTQ_FloatIntDiv          1002b5d4 f   srvclkm:sgxtransfer_utils.obj
 0001:0002a5f4       WriteEndOfRenderUSSECode   1002b5f4 f   srvclkm:pixevent.obj
 0001:0002a624       WriteEndOfTileUSSECode     1002b624 f   srvclkm:pixevent.obj
 0001:0002a6e4       PDSGeneratePixelEventProgram 1002b6e4 f   srvclkm:pds.obj
 0001:0002a784       CreateCCB                  1002b784 f   srvclkm:sgxutils_client.obj
 0001:0002a8d8       DestroyCCB                 1002b8d8 f   srvclkm:sgxutils_client.obj
 0001:0002aa08       _DllMainCRTStartup         1002ba08 f   corelib0:pegdmain.obj
 0001:0002aa38       __GSHandlerCheckCommon     1002ba38 f   corelib0:gshandler.obj
 0001:0002aa74       __GSHandlerCheck           1002ba74 f   corelib0:gshandler.obj
 0001:0002aa98       __security_init_cookie     1002ba98 f   corelib0:seccinit.obj
 0001:0002aaf4       __security_check_cookie    1002baf4 f   corelib0:armsecgs.obj
 0001:0002ab08       __gsfailure                1002bb08 f   corelib0:armsecgs.obj
 0001:0002ac14       _cexit                     1002bc14 f   corelib0:cexit.obj
 0001:0002ac30       _initterm                  1002bc30 f   corelib0:crt0dat.obj
 0001:0002ac64       _cinit                     1002bc64 f   corelib0:crt0dat.obj
 0001:0002ac98       memset                     1002bc98 f   corelib1:COREDLL.dll
 0001:0002aca8       swprintf                   1002bca8 f   corelib1:COREDLL.dll
 0001:0002acb8       __C_specific_handler       1002bcb8 f   corelib1:COREDLL.dll
 0001:0002acc8       free                       1002bcc8 f   corelib1:COREDLL.dll
 0001:0002acd8       malloc                     1002bcd8 f   corelib1:COREDLL.dll
 0001:0002ace8       memcpy                     1002bce8 f   corelib1:COREDLL.dll
 0001:0002acf8       swscanf                    1002bcf8 f   corelib1:COREDLL.dll
 0001:0002ad08       ??2@YAPAXI@Z               1002bd08 f   corelib1:COREDLL.dll
 0001:0002ad18       ??3@YAXPAX@Z               1002bd18 f   corelib1:COREDLL.dll
 0001:0002ad28       _purecall                  1002bd28 f   corelib1:COREDLL.dll
 0001:0002ad38       memmove                    1002bd38 f   corelib1:COREDLL.dll
 0001:0002ad48       calloc                     1002bd48 f   corelib1:COREDLL.dll
 0001:0002ad58       _XcptFilter                1002bd58 f   corelib1:COREDLL.dll
 0001:0002ad68       __security_gen_cookie2     1002bd68 f   corelib1:COREDLL.dll
 0001:0002ad78       __report_gsfailure         1002bd78 f   corelib1:COREDLL.dll
 0001:0002ad88       CreateEventW               1002bd88 f   coredll:COREDLL.dll
 0001:0002ad98       WaitForSingleObject        1002bd98 f   coredll:COREDLL.dll
 0001:0002ada8       GetTickCount               1002bda8 f   coredll:COREDLL.dll
 0001:0002adb8       InterlockedCompareExchange 1002bdb8 f   coredll:COREDLL.dll
 0001:0002adc8       __GetUserKData             1002bdc8 f   coredll:COREDLL.dll
 0001:0002add8       DeviceIoControl            1002bdd8 f   coredll:COREDLL.dll
 0001:0002ade8       FormatMessageW             1002bde8 f   coredll:COREDLL.dll
 0001:0002adf8       GetLastError               1002bdf8 f   coredll:COREDLL.dll
 0001:0002ae08       CreateFileW                1002be08 f   coredll:COREDLL.dll
 0001:0002ae18       CloseHandle                1002be18 f   coredll:COREDLL.dll
 0001:0002ae28       TerminateProcess           1002be28 f   coredll:COREDLL.dll
 0001:0002af3c       __IMPORT_DESCRIPTOR_COREDLL 1002bf3c     coredll:COREDLL.dll
 0001:0002af50       __NULL_IMPORT_DESCRIPTOR   1002bf50     coredll:COREDLL.dll
 0002:00000000       __imp_OutputDebugStringW   1002d000     coredll:COREDLL.dll
 0002:00000004       __imp_NKDbgPrintfW         1002d004     coredll:COREDLL.dll
 0002:00000008       __imp_SetLastError         1002d008     coredll:COREDLL.dll
 0002:0000000c       __imp_RegCloseKey          1002d00c     coredll:COREDLL.dll
 0002:00000010       __imp_RegQueryValueExW     1002d010     coredll:COREDLL.dll
 0002:00000014       __imp_RegOpenKeyExW        1002d014     coredll:COREDLL.dll
 0002:00000018       __imp_AdvertiseInterface   1002d018     coredll:COREDLL.dll
 0002:0000001c       __imp_GetModuleFileNameW   1002d01c     coredll:COREDLL.dll
 0002:00000020       __imp_DisableThreadLibraryCalls 1002d020     coredll:COREDLL.dll
 0002:00000024       __imp_RegSetValueExW       1002d024     coredll:COREDLL.dll
 0002:00000028       __imp_RegCreateKeyExW      1002d028     coredll:COREDLL.dll
 0002:0000002c       __imp_LocalAlloc           1002d02c     coredll:COREDLL.dll
 0002:00000030       __imp_LocalFree            1002d030     coredll:COREDLL.dll
 0002:00000034       __imp_LocalReAlloc         1002d034     coredll:COREDLL.dll
 0002:00000038       __imp_VirtualFree          1002d038     coredll:COREDLL.dll
 0002:0000003c       __imp_CeSetExtendedPdata   1002d03c     coredll:COREDLL.dll
 0002:00000040       __imp_VirtualAlloc         1002d040     coredll:COREDLL.dll
 0002:00000044       __imp_CacheRangeFlush      1002d044     coredll:COREDLL.dll
 0002:00000048       __imp_memset               1002d048     corelib1:COREDLL.dll
 0002:0000004c       __imp_swprintf             1002d04c     corelib1:COREDLL.dll
 0002:00000050       __imp___C_specific_handler 1002d050     corelib1:COREDLL.dll
 0002:00000054       __imp_free                 1002d054     corelib1:COREDLL.dll
 0002:00000058       __imp_malloc               1002d058     corelib1:COREDLL.dll
 0002:0000005c       __imp___rt_udiv            1002d05c     corelib1:COREDLL.dll
 0002:00000060       __imp_memcpy               1002d060     corelib1:COREDLL.dll
 0002:00000064       __imp_swscanf              1002d064     corelib1:COREDLL.dll
 0002:00000068       __imp_??2@YAPAXI@Z         1002d068     corelib1:COREDLL.dll
 0002:0000006c       __imp_??3@YAXPAX@Z         1002d06c     corelib1:COREDLL.dll
 0002:00000070       __imp___rt_sdiv            1002d070     corelib1:COREDLL.dll
 0002:00000074       __imp__purecall            1002d074     corelib1:COREDLL.dll
 0002:00000078       __imp___divs               1002d078     corelib1:COREDLL.dll
 0002:0000007c       __imp___itos               1002d07c     corelib1:COREDLL.dll
 0002:00000080       __imp___adds               1002d080     corelib1:COREDLL.dll
 0002:00000084       __imp___stod               1002d084     corelib1:COREDLL.dll
 0002:00000088       __imp_pow                  1002d088     corelib1:COREDLL.dll
 0002:0000008c       __imp___dtos               1002d08c     corelib1:COREDLL.dll
 0002:00000090       __imp___muls               1002d090     corelib1:COREDLL.dll
 0002:00000094       __imp___subs               1002d094     corelib1:COREDLL.dll
 0002:00000098       __imp___stou               1002d098     corelib1:COREDLL.dll
 0002:0000009c       __imp___utos               1002d09c     corelib1:COREDLL.dll
 0002:000000a0       __imp___rt_sdiv64by64      1002d0a0     corelib1:COREDLL.dll
 0002:000000a4       __imp_memmove              1002d0a4     corelib1:COREDLL.dll
 0002:000000a8       __imp_calloc               1002d0a8     corelib1:COREDLL.dll
 0002:000000ac       __imp__XcptFilter          1002d0ac     corelib1:COREDLL.dll
 0002:000000b0       __imp___security_gen_cookie2 1002d0b0     corelib1:COREDLL.dll
 0002:000000b4       __imp___report_gsfailure   1002d0b4     corelib1:COREDLL.dll
 0002:000000b8       __imp_CreateEventW         1002d0b8     coredll:COREDLL.dll
 0002:000000bc       __imp_WaitForSingleObject  1002d0bc     coredll:COREDLL.dll
 0002:000000c0       __imp_GetTickCount         1002d0c0     coredll:COREDLL.dll
 0002:000000c4       __imp_InterlockedCompareExchange 1002d0c4     coredll:COREDLL.dll
 0002:000000c8       __imp___GetUserKData       1002d0c8     coredll:COREDLL.dll
 0002:000000cc       __imp_DeviceIoControl      1002d0cc     coredll:COREDLL.dll
 0002:000000d0       __imp_FormatMessageW       1002d0d0     coredll:COREDLL.dll
 0002:000000d4       __imp_GetLastError         1002d0d4     coredll:COREDLL.dll
 0002:000000d8       __imp_CreateFileW          1002d0d8     coredll:COREDLL.dll
 0002:000000dc       __imp_CloseHandle          1002d0dc     coredll:COREDLL.dll
 0002:000000e0       __imp_TerminateProcess     1002d0e0     coredll:COREDLL.dll
 0002:000000e4       \177COREDLL_NULL_THUNK_DATA 1002d0e4     coredll:COREDLL.dll
 0002:000000e8       ?_rgbIdentity@@3PAUtagPALETTEENTRY@@A 1002d0e8     mode.obj
 0002:000004e8       ?EGPEFormatToPVR2D@@3PAHA  1002d4e8     mode.obj
 0002:00000510       ?gBitMasks@@3PAKA          1002d510     sgxmain.obj
 0002:0000053c       ?gaMix@@3PAEA              1002d53c     gpe:ddi_if.obj
 0002:00000980       ?gulGamma@@3KA             1002d980     gpe:rctblt.obj
 0002:00000984       ?szGamma@@3PAGA            1002d984     gpe:rctblt.obj
 0002:000009a8       ?szGammaValue@@3PAGA       1002d9a8     gpe:rctblt.obj
 0002:000009c0       ?alAlpha@@3PAJA            1002d9c0     gpe:rctblt.obj
 0002:000009e0       ?ajGammaCT_10@@3PAEA       1002d9e0     gpe:rctblt.obj
 0002:00000ae0       ?ajGammaCT_11@@3PAEA       1002dae0     gpe:rctblt.obj
 0002:00000be0       ?ajGammaInvCT_11@@3PAEA    1002dbe0     gpe:rctblt.obj
 0002:00000ce0       ?ajGammaCT_12@@3PAEA       1002dce0     gpe:rctblt.obj
 0002:00000de0       ?ajGammaInvCT_12@@3PAEA    1002dde0     gpe:rctblt.obj
 0002:00000ee0       ?ajGammaCT_13@@3PAEA       1002dee0     gpe:rctblt.obj
 0002:00000fe0       ?ajGammaInvCT_13@@3PAEA    1002dfe0     gpe:rctblt.obj
 0002:000010e0       ?ajGammaCT_14@@3PAEA       1002e0e0     gpe:rctblt.obj
 0002:000011e0       ?ajGammaInvCT_14@@3PAEA    1002e1e0     gpe:rctblt.obj
 0002:000012e0       ?ajGammaCT_15@@3PAEA       1002e2e0     gpe:rctblt.obj
 0002:000013e0       ?ajGammaInvCT_15@@3PAEA    1002e3e0     gpe:rctblt.obj
 0002:000014e0       ?ajGammaCT_16@@3PAEA       1002e4e0     gpe:rctblt.obj
 0002:000015e0       ?ajGammaInvCT_16@@3PAEA    1002e5e0     gpe:rctblt.obj
 0002:000016e0       ?ajGammaCT_17@@3PAEA       1002e6e0     gpe:rctblt.obj
 0002:000017e0       ?ajGammaInvCT_17@@3PAEA    1002e7e0     gpe:rctblt.obj
 0002:000018e0       ?ajGammaCT_18@@3PAEA       1002e8e0     gpe:rctblt.obj
 0002:000019e0       ?ajGammaInvCT_18@@3PAEA    1002e9e0     gpe:rctblt.obj
 0002:00001ae0       ?ajGammaCT_19@@3PAEA       1002eae0     gpe:rctblt.obj
 0002:00001be0       ?ajGammaInvCT_19@@3PAEA    1002ebe0     gpe:rctblt.obj
 0002:00001ce0       ?ajGammaCT_20@@3PAEA       1002ece0     gpe:rctblt.obj
 0002:00001de0       ?ajGammaInvCT_20@@3PAEA    1002ede0     gpe:rctblt.obj
 0002:00001ee0       ?ajGammaCT_21@@3PAEA       1002eee0     gpe:rctblt.obj
 0002:00001fe0       ?ajGammaInvCT_21@@3PAEA    1002efe0     gpe:rctblt.obj
 0002:000020e0       ?ajGammaCT_22@@3PAEA       1002f0e0     gpe:rctblt.obj
 0002:000021e0       ?ajGammaInvCT_22@@3PAEA    1002f1e0     gpe:rctblt.obj
 0002:000022e0       ?gaOutTable@@3PAU_F_RGB@@A 1002f2e0     gpe:rctblt.obj
 0002:000024b8       ?pfnDrvGradientFill@@3P6AHPAU_SURFOBJ@@PAU_CLIPOBJ@@PAU_XLATEOBJ@@PAU_TRIVERTEX@@KPAXKPAU_RECTL@@PAU_POINTL@@K@ZA 1002f4b8     gpe:rdrvgradfill.obj
 0002:000024c0       ?gulDither32@@3PAKA        1002f4c0     gpe:rdrvgradfill.obj
 0002:00002500       ?gDitherMatrix16x16Halftone@@3PAEA 1002f500     gpe:rdrvgradfill.obj
 0002:00002600       ?gDitherMatrix16x16Default@@3PAEA 1002f600     gpe:rdrvgradfill.obj
 0002:00002700       ?vTranslateIdentity@@3PAEA 1002f700     gpe:rdrvgradfill.obj
 0002:00002800       ?DefaultSaturationTable@@3PAEA 1002f800     gpe:rdrvgradfill.obj
 0002:00002980       ?Saturation16_5@@3PAEA     1002f980     gpe:rdrvgradfill.obj
 0002:000029c0       ?Saturation16_6@@3PAEA     1002f9c0     gpe:rdrvgradfill.obj
 0002:00002a40       ?pfnDrvAlphaBlend@@3P6AHPAU_SURFOBJ@@0PAU_CLIPOBJ@@PAU_XLATEOBJ@@PAU_RECTL@@3PAUtagBLENDOBJ@@@ZA 1002fa40     gpe:drvalphablend.obj
 0002:00002a48       ?g_pdwAnyBltPCode@@3PAKA   1002fa48     gpe:genblt.obj
 0002:0000bca0       pbtransferqueue_use        10038ca0     srvclkm:sgxtransfer_context.obj
 0002:0000c280       __security_cookie          10039280     corelib0:seccinit.obj
 0002:0000c284       __security_cookie_complement 10039284     corelib0:seccinit.obj
 0002:0000c288       ?gGPE@@3PAVGPE@@A          10039288     sgxmain.obj
 0002:0000c290       PATHOBJ_vGetBounds         10039290     gpe:ddi_if.obj
 0002:0000c294       PATHOBJ_bEnum              10039294     gpe:ddi_if.obj
 0002:0000c298       PALOBJ_cGetColors          10039298     gpe:ddi_if.obj
 0002:0000c29c       CLIPOBJ_bEnum              1003929c     gpe:ddi_if.obj
 0002:0000c2a0       EngGetPaletteFromPool      100392a0     gpe:ddi_if.obj
 0002:0000c2a4       EngAddPaletteToPool        100392a4     gpe:ddi_if.obj
 0002:0000c2a8       BRUSHOBJ_pvAllocRbrush     100392a8     gpe:ddi_if.obj
 0002:0000c2ac       BRUSHOBJ_pvGetRbrush       100392ac     gpe:ddi_if.obj
 0002:0000c2b0       CLIPOBJ_cEnumStart         100392b0     gpe:ddi_if.obj
 0002:0000c2b4       XLATEOBJ_cGetPalette       100392b4     gpe:ddi_if.obj
 0002:0000c2b8       PATHOBJ_vEnumStart         100392b8     gpe:ddi_if.obj
 0002:0000c2bc       EngCreatePalette           100392bc     gpe:ddi_if.obj
 0002:0000c2c0       EngCreateDeviceSurface     100392c0     gpe:ddi_if.obj
 0002:0000c2c4       EngDeleteSurface           100392c4     gpe:ddi_if.obj
 0002:0000c2c8       EngCreateDeviceBitmap      100392c8     gpe:ddi_if.obj
 0002:0000c2cc       EngReleasePooledPalette    100392cc     gpe:ddi_if.obj
 0002:0000c2d0       pfnGetGPEPerCard           100392d0     gpe:ddi_if.obj
 0002:0000c2d4       g_hmodDisplayDll           100392d4     gpe:ddi_if.obj
 0002:0000c2d8       ?g_pxlo@@3PAU_XLATEOBJ@@A  100392d8     gpe:ddi_if.obj
 0002:0000c2e8       ?uBCacheCT@@3KA            100392e8     gpe:rctblt.obj
 0002:0000c2ec       ?uFCacheCT@@3KA            100392ec     gpe:rctblt.obj
 0002:0000c2f0       ?aulCacheCT@@3PAKA         100392f0     gpe:rctblt.obj
 0002:0000c4bc       ?sizeCacheCT@@3KA          100394bc     gpe:rctblt.obj
 0002:0000c4c0       ?uGammaCacheCT@@3KA        100394c0     gpe:rctblt.obj
 0002:0000c4fc       ?gbHateMmx@@3HA            100394fc     gpe:rctblt.obj
 0002:0000c508       ?gMaskedConverter@@3PAVMaskColorConverter@@A 10039508     gpe:swconvrt.obj
 0002:0000c698       ?gLookupConverter@@3PAVLookupColorConverter@@A 10039698     gpe:swconvrt.obj
 0002:0000d6e8       ?gMonoConverter@@3PAVMonoColorConverter@@A 1003a6e8     gpe:swconvrt.obj
 0002:0000d710       ?gMaskedLRU@@3VLRU@@A      1003a710     gpe:swconvrt.obj
 0002:0000d724       ?gLookupLRU@@3VLRU@@A      1003a724     gpe:swconvrt.obj
 0002:0000d738       ?gMonoLRU@@3VLRU@@A        1003a738     gpe:swconvrt.obj
 0002:0000d74c       ?gGroupLRU@@3VLRU@@A       1003a74c     gpe:swconvrt.obj
 0002:0000d760       ?gGroupConverter@@3PAVGroupColorConverter@@A 1003a760     gpe:swconvrt.obj
 0002:0000e5d0       ?pfnGetAAMaskBits@@3P6AXPAK00@ZA 1003b5d0     gpe:aablt.obj
 0002:0000e858       ?g_BltFnPData@@3U_xpdata@@A 1003b858     gpe:genblt.obj
 0002:0000e8e0       ?g_CpuFuncs@@3UGenBltCpuFuncs@@A 1003b8e0     gpe:genblt.obj
 0002:0000e8fc       ?g_pPCodeRegisters@@3PAUPCodeRegisters_t@@A 1003b8fc     gpe:genblt.obj
 0002:0000e900       ?g_BltClock@@3KA           1003b900     gpe:genblt.obj
 0002:0000e904       ?g_fUseFastBlt@@3HA        1003b904     gpe:FastBlt.obj
 0002:0001012c       _exitflag                  1003d12c     corelib0:cexit.obj
 0002:00010130       __onexitend                1003d130     <common>
 0002:00010134       __onexitbegin              1003d134     <common>
 0002:00010138       _pRawDllMain               1003d138     <common>

 entry point at        0001:0002aa08

 Static symbols

 0001:00003928       ?ConvertStringToGuid@@YAHPBGPAU_GUID@@@Z 10004928 f   power.obj
 0001:0000f280       ?GetNearestIndex@@YAKK@Z   10010280 f   gpe:rctblt.obj
 0001:0001267c       ?GetAAMaskInfo@@YAXH@Z     1001367c f   gpe:aablt.obj
 0001:000127dc       ?InitGamma@@YAXXZ          100137dc f   gpe:aablt.obj
 0001:00013880       ?MDiv64@@YA_J_J00@Z        10014880 f   gpe:rdrvgradfill.obj
 0001:00015620       ?RectFillBlt@@YAHPAU_SURFOBJ@@PAU_DRVGRADIENTRECTDATA@@P6AXPAVGPESurf@@1@Z@Z 10016620 f   gpe:rdrvgradfill.obj
 0001:000157ec       ?GFGetShift@@YAXKPAK0@Z    100167ec f   gpe:rdrvgradfill.obj
 0001:0001f840       AltBltClipped              10020840 f   libpvr2d:pvr2dblt.obj
 0001:0002038c       InitDisplayDevice          1002138c f   libpvr2d:pvr2dinit.obj
 0001:00020f20       PrepareNormalBlit          10021f20 f   srvclkm:sgxtransfer_queue.obj
 0001:00022308       PrepareTextureUpload       10023308 f   srvclkm:sgxtransfer_queue.obj
 0001:000229bc       PrepareMipGen              100239bc f   srvclkm:sgxtransfer_queue.obj
 0001:00022fc4       PrepareFillOp              10023fc4 f   srvclkm:sgxtransfer_queue.obj
 0001:000236ac       PrepareBufferBlt           100246ac f   srvclkm:sgxtransfer_queue.obj
 0001:00023d24       PrepareCustomOp            10024d24 f   srvclkm:sgxtransfer_queue.obj
 0001:00023fb8       PrepareFullCustomOp        10024fb8 f   srvclkm:sgxtransfer_queue.obj
 0001:000241dc       PrepareCustomShaderBlit    100251dc f   srvclkm:sgxtransfer_queue.obj
 0001:00024914       PrepareClipBlit            10025914 f   srvclkm:sgxtransfer_queue.obj
 0001:00024e38       PrepareColourLUTBlit       10025e38 f   srvclkm:sgxtransfer_queue.obj
 0001:000254f0       SGXSubmitTransfer          100264f0 f   srvclkm:sgxtransfer_queue.obj
 0001:00026bc4       TQAllocUSEFrag             10027bc4 f   srvclkm:sgxtransfer_context.obj
 0001:00026eb4       TQCreatePDSPrimFrag        10027eb4 f   srvclkm:sgxtransfer_context.obj
 0001:00026fe0       TQCreatePDSSecondaryFrag   10027fe0 f   srvclkm:sgxtransfer_context.obj
 0001:0002718c       TQCreateHWBGObject         1002818c f   srvclkm:sgxtransfer_context.obj
 0001:00027270       TQCreateFast2DISPControlStream 10028270 f   srvclkm:sgxtransfer_context.obj
 0001:00027340       TQCreatePixelEventProgram  10028340 f   srvclkm:sgxtransfer_context.obj
 0001:000290b4       SGXTQ_PatchPDSProgram      1002a0b4 f   srvclkm:sgxtransfer_utils.obj
 0001:0002a90c       _DllMainCRTStartupHelper   1002b90c f   corelib0:pegdmain.obj
 0001:0002ab4c       doexit                     1002bb4c f   corelib0:cexit.obj
 0001:0002ae38       ??__EgGroupConverter@@YAXXZ 1002be38 f   gpe:swconvrt.obj
